:0A00000026C0FECFFDCFFCCFFBCFE2
:10000A00FACF3FC0F8CFF7CFF6CFF5CFF4CFF3CF83
:10001A00F2CFF1CFF0CFEFCFEECFEDCFD714CD5D4A
:10002A001E5BDB15DF5F080F008B98FCCB88A800EE
:10003A00F7EFDFBF6400C80090012003F8FFFCFF60
:10004A00FEFFFFFFF894EE27ECBBE5BFF8E1A4B78B
:10005A00A77FA4BFF1BDE1BD8DE0A2E0ED938A9533
:10006A00E9F780E8A0E6ED938A95E9F7E0E0E3BBDB
:10007A00E0E0E4BBE0E0E5BBEFEDEDBFC0E8D0E0D7
:10008A000DC10A92AA93EA93FA93EFB7EA93E2B3FD
:10009A00E867E2BBA9E8A30DEC9106D2EA5DFF4F3F
:1000AA00049008BAE2B3AE2FE32DFED1E65CFF4F0F
:1000BA00E491EA23E2BBA0E09899A1E0A13019F407
:1000CA00E1E0E31509F001C0C59A3394E4E03E1675
:1000DA0008F03324E991EFBFF991E991A9910990C8
:1000EA0018956AD3EDB7EA931F93EDB7EA930F9386
:1000FA00EDB7EA933F93A1D13F910F911F91E8EB9E
:10010A00FBE0D4D1EDB7EA931F93EDB7EA930F93CF
:10011A00EDB7EA932F9391D12F910F911F91231746
:10012A0021F4C7D1C6D1C5D19DD159C045D3EDB7A8
:10013A00EA931F93EDB7EA930F93EDB7EA933F93D0
:10014A007CD13F910F911F911F3F09F0212E0F3F44
:10015A0009F0702EE22DB0D1E0938900E22DEF7004
:10016A00AED1E72DA9D1E0938B00E72DEF70E09394
:10017A008C0035C021D3809918C000E010E01A30F5
:10018A0038F4E1E0F0E092D1809B0F5F1F5FF7CF78
:10019A00063058F02A9273D13E2F3F5F383108F06B
:1001AA0030E03A9378D12E2E8DD1819918C000E093
:1001BA0010E01A3038F4E1E0F0E078D1819B0F5F6B
:1001CA001F5FF7CF063058F07A9259D13E2F3F5F22
:1001DA003C3308F030E03A935ED17E2E73D1F3D2ED
:1001EA00249608952497E6D2A201002440145004CC
:1001FA0014F0ECE006C0FA01E095F0953196AF01F3
:10020A00EAE0E0938900EBE0E0938C00989AFA0127
:10021A00A4D2E887F987FA01EF70F070EE83FF83C2
:10022A001885AE81BF81EAE0F0E0B0D296D20E2FF7
:10023A001A9331D13E2F143638F4A0918900AA308E
:10024A0011F41A3008F408C09898E32F35D137D141
:10025A00E32FEF70E0938B00A0918900AA3011F48C
:10026A001A3008F004C0EAE81083EBE80083A09192
:10027A008900AC3011F4143608F00DC0E32F1CD1FC
:10028A00E03021F0E32F18D1E0938900E32FEF70DB
:10029A0016D1EBE8008395D22A960895E0E8E6BDE8
:1002AA00E0E0E6BDEABBEBBBEFEFE7BBE0E0E8BBB3
:1002BA00E8E7E1BBEBEFE2BBE0E0E0BFE3BFE2BFB0
:1002CA00E6BFECBFE0BFE3E0E3BFE0E0EBBFE5BFC2
:1002DA00E2E0E9BFE0E0EDB9E0E8E8B969D1E0EFD2
:1002EA00EA93EDE8EA93B4D10E2F7894EDE0E09327
:1002FA008900EEE0E4D0EFE0E0938B00ECE80083C5
:10030A00ECEDF5E0D3D0EDDE10E0143160F40EDF51
:10031A00989902C0989A01C098982CDFE4EFF1E00E
:10032A00C5D01F5FF2CF0130A0F010E0101788F49B
:10033A00E12F1F5FA9E01FD2E357EA934BD02F01A9
:10034A00C5D0E415F50509F04DDFE0EDF7E0AED0D4
:10035A00EDCFDACFFFCF1A932BD1E03011F4E0E0E2
:10036A0069C0E981E03079F0F894E5E5B2D0789493
:10037A0010E0F894A981ED91A983ABD078941F5F1E
:10038A001830B8F304C0F894ECECA3D07894E1E008
:10039A0051C014D2EA81EA93DEDFE03019F4E0E0DA
:1003AA0014D26BC0F894EEEB94D0789410E000E885
:1003BA00F8940F930F5F3DD1AF91EC9378941F5F40
:1003CA001930B0F3E0E8EA93E9E0EA93B0D1CED18C
:1003DA00FCD153C01A937FD0DCDFE03011F476D021
:1003EA0029C0E0918400E295EF70E695E3701E2F34
:1003FA0072D0B1DFE03011F469D01CC0F894E4E4A3
:10040A0068D07894E12FAEE3B0E068D04FD063D0E3
:10041A00C0DFE03011F45AD00DC0F894C9D07894F6
:10042A00E12FA6E4B0E05AD0A0918000B0918100FB
:10043A00EA23FB2318812296089557D094D05FD0DF
:10044A00E1EDEA9390D0E1E0EA9372D0A881EC93CF
:10045A00E1E0EA936DD0A981EC932BD069D0AA810F
:10046A00EC930AC042D07FD0E881EA937CD033D0A3
:10047A007AD0EA81EA9377D051D023960895E88119
:10048A00E295EF70AE2FAA0FAA0FEA0FEE0FA9910D
:10049A00AF70EA0F0895A991EE27AA5012F0E05F13
:1004AA00FCCFA65FEA0F0895F0E00895FA93EA9365
:1004BA0073C0E0E0EA930895E295EF700895E0933F
:1004CA008A0008952A927A926A92CCCFE1EFF8EDE7
:1004DA000895EA93B3C0E981EA930895E5DFEE0F40
:1004EA00FF1FEA0FFB1F62D1089509D0E0EDEA93DE
:1004FA003AD0DFCFD898D998D09AD19815C0D19848
:10050A00D098EE270000C99B0895C89B089504D08F
:10051A00D19A02D0D09AE1E067E007C0D19AD09A86
:10052A0003D0D098F9DFD1986DE06A95F1F7089574
:10053A0078E0D098F1DFC89BFECFEEDF8894C999A6
:10054A000894D09AF1DFEE1F7A9599F7799177237B
:10055A0011F4D19801C0D19ADFDFD098E5DFD09AA3
:10056A00DBDFD198D9CFE99178E0EE0F10F4D1987A
:10057A0001C0D19AD9DFD098CFDFC89BFECFCCDF9C
:10058A00D09A7A9591F7D198C7DFD098CDDFE1E07C
:10059A00C999EE27D09A0895E991F991309639F0E0
:1005AA0088EE93E00197F1F7A8953197C9F7089576
:1005BA00EE2792988A9A80EE91E00197F1F78A984D
:1005CA0083E18A95F1F7829B089585E68A95F1F78A
:1005DA00829BE39586E891E00197F1F708958A9A5C
:1005EA0083E08A95F1F78A988FE08A95F1F78894E3
:1005FA0082990894E7958BE68A95F1F70895E8942D
:10060A008A9A83E08A95F1F770FD8A9881E18A9542
:10061A00F1F7829903C070FF03C0089570FF08952F
:10062A0084E68A95F1F78A9887E08A95F1F76894C3
:10063A00089568E0D4DF6A95E9F7089568E079914A
:10064A00EE27DDDF26F477956A95D9F7E3950895C5
:10065A004F935F9311244427A881BB27012C1124AF
:10066A00A7DFEE23F9F0E981EA93E8DF51E05015BC
:10067A0098F4B5DFE7FD08C0B2DFE7FD06C03FD05A
:10068A00892319F4152E01C0AADF39D0892370E015
:10069A0009F071E0B4DF1EC0A2DFE7FF0BC09FDFE5
:1006AA00E7FF05C0E42F5F914F9122960895689461
:1006BA0036D0EFCF94DFE7FF01C003C0501531F009
:1006CA00152EE8942CD077279ADF04C0689427D097
:1006DA0071E095DF5395513454F281DFEE1FEE1F1E
:1006EA00E1701896EC93189743951120D9F259E0C6
:1006FA00EC911996EC9318975A95D1F7AFCFE52F4D
:10070A00EA956E2FE695E695E695EA0FFF27808132
:10071A0091E0677019F0990F6A95FCCF0895EFDFA1
:10072A001EF09095892301C0892B80830895EE27B6
:10073A008881882381F068E1A981BB2798E0FD912F
:10074A007F2F7E27779508F4E627E795F6959A9501
:10075A00B9F78A9599F722960895F695E795F69549
:10076A00E795F695E795F695E7950895EE23E1E086
:10077A0009F0EE2708950A2EAA1BB9E003C008F46F
:10078A00A00DA695E795BA95D1F708950A2E1B2EC6
:10079A0081E1AA27BB1B05C010F4A00DB11DB695B7
:1007AA00A795F795E7958A95B9F708950590F49175
:1007BA00E02D08955A934A933A932A931A930A93E7
:1007CA0008955D814C813B812A81198108810895B0
:00000001FF
